:1000000050230D30840084280B1D09009000030E3E
:100010008F008312051C0E2891011328110F9100E7
:100020004120FF309C00851C172892011C28120FCC
:1000300092004120FF309C00051D202893012328B9
:10004000130F930041201A081B0403192C289B0F3F
:100050002C289A0F2C289D151708031D9703180AA2
:10006000031935281808031D98031C0803193B2899
:100070009C0B3B281D160F0E8300900E100E0B11CB
:100080000900FB309A00B4309B000800820754340A
:100090005834003452345834003455344E3400341B
:1000A0004C344F3443344B344534443400342034DE
:1000B00020340034203444344934533450344C34E4
:1000C00041345934203400344D3455344C34543494
:1000D00000344D344134583400344D3449344E34B6
:1000E000203400342034563443344F3420344F34D9
:1000F00046344634533445345434203400342034A8
:100100004D3448347A34003443308C008001840A02
:100110008C0B86288316173085000130860004304A
:10012000810083128101A0308B00FE30860085158E
:100130000D22051D9D16742341209D11E421583088
:10014000DB21D821D8218A30E5210930EB21C030CC
:10015000E521DA2180219D199C2880238030E5212A
:10016000051EB7281D1F9D171D175230BB281D1BCC
:100170009D171D135430DB218830E52106301D1DED
:10018000C4281F1FC4281030EB219D1FCA289C1BA8
:10019000E2289D131D1FD72824303B2358232830E5
:1001A000492334232A30492327232430E1282630C9
:1001B0003B2358232E30492334233030492327232F
:1001C00026304223C42193219D1EAB28DD23191C18
:1001D000AB28DF211330EB211D30EB219D199C282A
:1001E000C421AE231918A30ABF231918A303013091
:1001F00023020318FD280130A30015302302031C3D
:1002000003291430A300C2012308C3000A304302AB
:10021000031C0D29C300C20A06298E30E5214208BD
:10022000303EDB214308303EDB21A523191CEE289C
:10023000E4212630EB210330EB211330EB21802128
:100240009D199C28C42128308821283042239321DD
:10025000A523191C2029E4212230EB219D199C287B
:10026000C4212A303B235823283086212A304223B8
:100270009321A523191C2E29E4210330EB212B30D7
:10028000EB219D199C28C4212C30B3212C30422312
:100290009321A523191C4129E4212630EB210030AC
:1002A000EB211330EB219D199C28C4212E3088218D
:1002B0002E3042239321A523191C5329E4212230F7
:1002C000EB219D199C28C42130303B2358232E302C
:1002D0008621303042239321A523191C6129E42172
:1002E0000030EB212B30EB219D199C28C4213230AA
:1002F000B321323042239321A523191C74299C2851
:10030000CA30E5213830EB21D921080049238C2956
:100310003B235823B901BA0134239430B90070301B
:10032000BA00272308009D103709C039031D9F29F3
:100330009D14B709B8090130B8070318B70A230894
:10034000B6000310B60DB60DB607F0229822C130E4
:10035000E5214130840009308C000008DB21840A4B
:100360008C0BAD2908003B238030B7065823A730FB
:10037000B9001030BA0027235830B900F030BA0065
:1003800034238030B70608004722051ECD292430CB
:100390003B23213042232C30D22926303B232130ED
:1003A0004223323049231023232221303B230800EB
:1003B000DA21DA212030A100A2008614F4290130CC
:1003C000E5211830512308008130A100A2008610D9
:1003D000F42186140800A0004620FF390319080004
:1003E000DB212008013EEB2906118316013086002F
:1003F00083128615F030A10506080E392104860007
:1004000086118615A20EF030A20506080E392204C8
:10041000860086114B309422080086011E221E227F
:100420001E2228308600861150232830E52108300E
:10043000E521DF210630E5210C30E5295023383055
:100440008600861108009E101D156D230330B9002B
:10045000E830BA0034236D30B9006030BA00272389
:10046000343049231E230319442A3430422379228D
:10047000C2306B2237086B2238086B22AE306B22F9
:10048000FF306B227E221F139E181D1108001F1FB4
:100490004D2A1808031D5F2A68227922C3306B2277
:1004A00008308C00932286149322060C9F0D861030
:1004B0008C0B522A8F2285227E221F1B6822051E4A
:1004C0001F1F662A1D1D662A851108008515080054
:1004D0006E3098000800A00008308C00A00D0318B2
:1004E0008F22031C8A2285228C0B6E2A8F22852262
:1004F000080086148F2293228A22872A8A22932236
:10050000861493228F22932208009322861493222A
:100510008610080006108316061083120800831642
:100520000614831208000F308D008D0B952A0800E9
:10053000031018308C00C201C401C601C901BF0DEF
:10054000BE0DBD0DC90DC60DC40DC20D8C0BCB2A41
:10055000490EC800460EC500440EC300420EC1003D
:100560001D104130E0224230E0224330E02244308E
:10057000E0224530E0221D144630E022A530C700BD
:100580004830E0224930E0229D1C080040088400E9
:100590002D30800008004930D4224630D422443027
:1005A000D4224230D4229F2A840003300007A000C6
:1005B000A019800030300007A000A01B80000800B8
:1005C00084000F3000050319E92A303E80001D1415
:1005D00008001D18E52A203080000408C00008002B
:1005E000BF013708BD003808BE0008308C00B60CCB
:1005F0000318FF2A8C0BF72ABD01BE010800031067
:100600000A2BB60C031C0A2B3808BE073708031840
:10061000370FBD07BD0CBE0CBF0C8C0B012B0800A7
:100620003A08B80739080318390FB70708003A081D
:10063000B8023908031C390FB70208003A0838021B
:10064000A0003908031C390A3702200408003908C1
:10065000BB003A08BC000130BA070318B90A1E23D0
:10066000031C08003B30382B1E23031808003930C8
:100670003B239E14080084000008B700840A000889
:10068000B8000800840037088000840A3808800019
:10069000080084000008B900840A0008BA000800B5
:1006A00076308D008E018E0B532B8D0B532B080053
:1006B000B9010130051D1430BA00B62319181023F2
:1006C000C723191817230230051DC830BA00AE23FE
:1006D00019181023BF23191817233709C039031D10
:1006E0000800B701B80108008901233084001130E7
:1006F0008C0093238000890A840A8C0B792B0800D4
:100700001D1E08001D1289012330840011308C0049
:100710009323000203198E2B00089823890A840A68
:100720008C0B882B08008316081483120808080015
:10073000880083160812081555308900AA308900F0
:100740008814081EA12B831208001E30A000160872
:1007500099001302D0231308960008006430110298
:10076000031CB62B463091006630B72B3C30A000FE
:10077000140899001102D023110894000800643075
:100780001202031CC72B463092006630C82B3C3047
:10079000A000150899001202D02312089500080045
:1007A0000318DA2B1908053C0318DA2B1908200264
:1007B000FF30031C030199000800A523191C080041
:0E07C00017080319E42B080019309700DA2BF4
:02400E00FB3F76
:104200000100000019000000190000001800000063
:104210001A00000000000000180000001A00000052
:0242200000009C
:00000001FF
